:10000000830100308A003D28DB0003088301DC0007
:1000100083122A088100A90AAB0A1F30AB05003001
:100020008A002B08162086000B1137288207083417
:1000300009340A340C340D340E340E340F340F34BA
:100040000F340E340E340D340C340A3409340834B1
:1000500006340534033402340134013400340034EE
:10006000003401340134023403340534063483127D
:100070005C088300DB0E5B0E0900213084005130E8
:100080005320203084002130532083010730DA00D0
:10009000F830D90051308400593057208301392D70
:1000A00004068001840A0406031D50280034F00071
:1000B00062208000840A040870060319003458285E
:1000C0008312D900DA1B6B285A088A005908D90A0A
:1000D0000319DA0A820083135A1883175908D90AB8
:0600E00084000008080086
:100654008312DD232C3A8312031908002B2B8316F3
:100664009B001C148312CF0083161A0883120800FF
:10067400F0000030711870070310F00D0310F10C36
:10068400F108031908003C2BF401F5010310F30CE5
:10069400F20C031C542B7008F40771080318710A38
:1006A400F5070310F00DF10D7208730403190034FB
:1006B400482B8511A01985158312CF000A30CE006E
:1006C4005130AE00861F6A2B5930AE07AE0B682B33
:1006D400640083124F1C732B8515A01D772B851185
:1006E400772B8511A01D772B851503148312CF0C4E
:1006F400CE0B622B0800CD01CE01CF01D0009F2B81
:100704000A30F200F3014E08F1004D08F0004623D0
:100714004F08500784000008F000F1017408F00746
:100724000318F10A7508F107D0307007CD00FF30C7
:10073400031800307107CE00CF0A033083124F0232
:10074400031C822B4E08F1004D08F00008004130D4
:100754005B2354305B2309305B230230CF2BDD2332
:10076400CD0083169C18B42B83124D0883169B006E
:100774008312DD2383169A0003108B1B03148B133F
:1007840083161C1555309D00AA309D009C141C1125
:1007940003188B1783124D0831235B238312DD2347
:1007A400CD00573A0319B12B83124D08523A031D59
:1007B4000800DD23CE2BE52B6400061A061FE42B6C
:1007C4000510E62B05148312051AEA2BA019DE2B5B
:1007D400051EEE2BA01DDE2BCE012830AE00AE0B85
:1007E400F12B0830CF0064008312861FFB2BAA3044
:0C07F400FC2B5130AE00AE0BFD2B0310AF
:100800008312CE0CA01D072C051A0A2C092C051EDC
:100810000A2CCE17CF0BF52B861F102CAA30112CCB
:100820005130AE00AE0B122C8312A019051E192CEC
:100830001C2CA01D051A1E2C0830A0064E0808000E
:10084000CF01D00008304F02831203180800201196
:10085000501820150310A01C422CA70CA80C201D1A
:10086000332C0130342C0030F000031C392C0130C3
:100870003A2C0030F0060319412C8430A7060830CA
:10088000A80603108312D00CA01E4C2C640020304C
:1008900029020318512C462C64003A302902031C0B
:1008A0004C2CA901201D692CAC0A201E722C2C088E
:1008B000053A031D722CA01E632C6400203029020F
:1008C0000318682C5D2C64003A302902031C632C49
:1008D000A901A01A6D2CCA306E2CE730AA00203076
:1008E000A006AC01CF0A08304F0203180800272CDD
:1008F000CD01CD0A8F2C6400061E061F832CCD016E
:10090000CD0A0514842C0510CE0120304E020318A8
:100910008E2CCE0A20304E02031C892CCD0A831265
:10092000CD08031D7B2C0515A0128316811581129D
:10093000C630831281008B17FF30A800A700A010DB
:100940001D303123CD008312CD080319AB2C0030AC
:100950002024CD03A32C7E302024A0142016AC012B
:10096000CD018312CD0A4D033123CE0020244E1C2D
:10097000B12C033083122024F03020242130202495
:10098000CD0108304D020318CD2C83124D08393E9D
:10099000840000082024CD0AC12C1E30831231238C
:1009A0002024CD0109304D020318DE2C83124D089E
:1009B000413E840000082024CD0AD22C1F3083122F
:1009C00031232024CD0103304D020318EF2C831274
:1009D0004D08513E840000082024CD0AE32C2F301E
:1009E00083122024CD0103304D020318FF2C831203
:1009F0004D08543E840000082024CD0AF32C2F30EB
:100A000083122024413020243D3020242608303E0B
:100A100020242508303E20242408303E20242308AA
:100A2000303E20242208303E20242108303E20245D
:100A3000203020242030CD008312CD0A4D033123F5
:100A4000CE00CE0883120319282D4E0820241C2D19
:100A5000A010FF30A806A706280820242708202475
:100A600020127E3020247E30202405118B13831227
:100A7000080064008B018B1607309F0083168113DA
:100A800010308500F03086008312061F492D0514B2
:100A90004A2D051085140511572D4A08213A031DCA
:100AA000572DA923572D4A08563A03195F2E640083
:100AB0008312DD23CA00243A031D4D2D8312DD234A
:100AC000473A031D572D8312DD23503A031D572D3E
:100AD000831202308506DD23CA00473A031D532DD9
:100AE0008312DD23473A031D572D8312DD23413A3C
:100AF000031D572D8312B70A0319B80A1C3031237E
:100B000000380319972D3C30F200F3011C303123DB
:100B1000F000F101462375083802031D912D740879
:100B20003702031C952D2014972D83122010831259
:100B3000861A20189C2D572DDD232A23DD23B9008A
:100B4000DD23BA00DD23BB00DD23BC00DD23BD00B7
:100B5000DD23BE00DD23BF002A23DD23C0002A23BE
:100B6000DD23C100DD23C200DD23C300DD23C4007B
:100B7000DD23C500DD23C600DD23C700DD23C8005B
:100B80002A23DD23C900DD23DD23303A0319CC2DD0
:100B900039082C3A031DD42DC430B707031CB80301
:100BA000061B572D0510572D8312061BD82D051433
:100BB000DD232A232A23A101A201A301A401A50167
:100BC000A601DD23CB00CA012D3A83120319592E49
:100BD0002508A6002408A5002308A4002208A300D5
:100BE0002108A2002130F1004B08D03E3A23CC006E
:100BF000643083124C02031C1D2E9C30CC07A20AC9
:100C00000A302202031CF82DF630A207A30A0A308C
:100C10002302031CF82DF630A307A40A0A3024028D
:100C2000031CF82DF630A407A50A0A302502031C80
:100C30001B2EF630A507A60AF82D0A30F1004C0845
:100C400088274A07A1000A302102031C462EF630ED
:100C5000A107A20A0A302202031C462EF630A20780
:100C6000A30A0A302302031C462EF630A307A40A67
:100C70000A302402031C462EF630A407A50A0A30C7
:100C80002502031C462EF630A507A60A83124C083F
:100C9000CA000A304A02031C502EF630CA07492EF9
:100CA000DD23CB002C3A0319582E4B082E3AE52DA4
:100CB0008312782420100230B700B801572D831218
:100CC000DD23543A031D572D8312DD23473A031DBC
:100CD000572D8312DD233030D200D300CA00831297
:100CE0005208D1005308D2004A08D300DD23CA00BD
:100CF0002E3A03197F2E4A082C3A031D6F2E8312B9
:100D0000DD234D3A8312031D802EDD233030D500C4
:100D1000D600CA0083125508D4005608D5004A08E8
:100D2000D600DD23CA002E3A03199A2E4A082C3A1F
:100D3000031D8A2E1C30831231230038031D572DCA
:100D400054307D237008B5007108B60051307D2302
:100D50007008B3007108B4004D303123F000F10188
:100D60007108803AF2003608803A7202031DBA2EEA
:100D700035087002031CCC2E3C308312F200F301C4
:100D80004C303123F000F10146237408B10075089E
:100D9000B200AF01B001482F483083123123AD00BB
:100DA0004E303123F000F1017108803AF20036082C
:100DB000803A7202031DDE2E350870020318E62EFB
:100DC0004B3083123123B100B201102F4E30831209
:100DD0003123F200F3014B303123F000F1014623BF
:100DE0007408F0007508F1003608F3003508F200C9
:100DF00073277408B1007508B2000A30F200F301DD
:100E000049303123F000F10146237408F0007508E1
:100E1000F1003608F3003508F20073277408AD07B7
:100E2000513083122D02031C172F5030AD00570A8A
:100E30000319580A031D202F3308D7003408D8009F
:100E400057083302AF005808031C580A3402B00098
:100E5000B01F322F33085702AF003408031C340A86
:100E60005802B0003008803AF00080307002B5308F
:100E700003192F02031C492F6830F0000130F100E4
:100E80002F087002AF003008031C300A7102B00056
:100E900083122D08F000F1017108803AF200300849
:100EA000803A7202031D562F2F0870020318652F17
:100EB0004A303123F000F10138087102031D622F1E
:100EC000370870028312031C6D2F38083202031D8D
:100ED0006B2F370831020318572D20143308D70021
:100EE0003408D800572DF601F11F7D2FF009F00AC4
:100EF0000319F103F1097617F61773088039F6061E
:100F0000F31FBF2FF209F20A0319F303F309BF2FEE
:100F1000F000F4010310FD307107031CAF2FF30143
:100F2000F0307105031D972F0430F300F10EF2012C
:100F30000310F30AF10D031C992FF10C71087002D4
:100F40000318F000F20DF30B9D2FF41FA92FF209E7
:100F5000F20A7208F41F0800F009F00A0800F10C08
:100F60000318B82FF10C031CF0010310F00C031C44
:100F700003107008F200F001F00DA52FF601F40146
:100F8000F50172087304031DC82FF001F10100344C
:100F90001F30F6040310F60AF20DF30D031CCB2FDD
:100FA000F30CF20C73087102031DD82F7208700243
:100FB000031CE02F7208F0027308031C730AF1028D
:100FC000F40DF50DF60BF61AD02FF61FEC2FF409E1
:100FD000F40A0319F503F5097408F2007508F30023
:100FE000761F0034F009F00A0319F103F109003407
:100FF000303430343034303430343034FF34FF3433
:02400E00663F0B
:104200008200A0008A00A400B000A20060009C0010
:104210009E0086008200980098006000A4008A003A
:1042200098008200B20040006000AE00920088005A
:104230008A00640040006500000032002F003E004C
:10424000000000000000000000000000000000006E
:10425000000000000000000000000000000000005E
:10426000000000000000000000000000000000004E
:10427000000000000000000000000000000000003E
:10428000000000000000000000000000000000002E
:0E4290001400190005005A001400030032004B
:00000001FF
